:1000000004EF00F0FFFFFFFFA9EC01F02E0E666E7B
:100010002E0E676E2E0E686E2E0E696E2E0E6A6E96
:100020002E0E6B6E2E0E6C6E2E0E6D6E2E0E6E6E76
:100030002E0E6F6E2E0E706E2E0E716E2E0E726E56
:100040002E0E736E2E0E746E2E0E756E766A200E48
:10005000776E4D0E786E690E796E6B0E7A6E720E3B
:100060007B6E6F0E7C6E430E7D6E200E7E6E310EAB
:100070007F6E380E0001806F460E816F320E826FE8
:10008000350E836F320E846F200E856F200E866FC3
:10009000876B4D0E886F650E896F730E8A6F2E0EFB
:1000A0008B6F520E8C6F410E8D6F300E8E6F200E47
:1000B0008F6F200E906F916B3D0E926F936B3D0E84
:1000C000946F956B3A0E966F200E976F986B4EEC6F
:1000D00005F0820E0001996F0F0E9A6F810E9B6FD3
:1000E0000F0E9C6FFCEC02F0020E0C6EFF0E0B6EFE
:1000F000FF0E0A6E0C2E01D007D00B2E01D003D0BC
:100100000A2EFED7FAD7F6D7060E0B6EFF0E0A6E32
:100110000B2E01D003D00A2EFED7FAD70A0E0A6E94
:100120000A2EFED7820E0001996F0F0E9A6F810E74
:100130009B6F0F0E9C6FFCEC02F0010E0001A36F91
:1001400025EC04F080821AC099F01BC09AF0660E6C
:1001500000019B6F000E9C6FAFEC04F000C01AF022
:1001600001C01BF0010E0001996F010E9A6F770E0E
:100170009B6F000E9C6FA6EC03F0809480920B0E98
:100180000C6EFF0E0B6EFF0E0A6E0C2E01D007D008
:100190000B2E01D003D00A2EFED7FAD7F6D7330E96
:1001A0000B6EFF0E0A6E0B2E01D003D00A2EFED767
:1001B000FAD7880E0A6E0A2EFED780848082010E3E
:1001C000A36F25EC04F0616A626A8280612A61C0D3
:1001D00099F0000E00019A6F1AC09BF01BC09CF0B2
:1001E0009BEC02F0010E0001996F010E9A6F1AC08C
:1001F0009BF01BC09CF0A6EC03F01AC099F01BC04A
:100200009AF0880E9B6F000E9C6FAFEC04F000C05C
:100210001AF001C01BF0010E0001996F070E9A6FD2
:1002200000C09BF001C09CF0A6EC03F0020E996F99
:10023000010E9A6F920E9B6F000E9C6FA6EC03F05E
:10024000996B87EC04F000C063F001C064F0820E8B
:100250000B6EFF0E0A6E0B2E01D003D00A2EFED7B6
:10026000FAD7870E0A6E0A2EFED7000063C099F0F7
:1002700064C09AF01AC09BF01BC09CF09BEC02F08B
:10028000020E0001996F010E9A6F940E9B6F000E83
:100290009C6FA6EC03F0D5EC04F0030E0C6EFF0E81
:1002A0000B6EFF0E0A6E0C2E01D007D00B2E01D064
:1002B00003D00A2EFED7FAD7F6D70B0E0B6EFF0E21
:1002C0000A6E0B2E01D003D00A2EFED7FAD7180ED5
:1002D0000A6E0A2EFED782903F0E6114006E00C097
:1002E00065F000C080FF020E0001996F080E9A6F42
:1002F000960E9B6F000E9C6FA6EC03F065C099F004
:100300001AC09AF01BC09BF052EC03F0D5EC04F03D
:10031000030E0C6EFF0E0B6EFF0E0A6E0C2E01D03C
:1003200007D00B2E01D003D00A2EFED7FAD7F6D76E
:100330008C0E0B6EFF0E0A6E0B2E01D003D00A2E10
:10034000FED7FAD7A10E0A6E0A2EFED700003DD7BF
:10035000FFD74D0E1C6E690E1D6E6B0E1E6E720E5B
:100360001F6E6F0E206E430E216E200E226E310E18
:10037000236E380E246E460E256E320E266E350E16
:10038000276E320E286E200E296E430E2A6E6F0ED7
:100390002B6E6E0E2C6E610E2D6E690E2E6E720E11
:1003A0002F6E200E306E4C0E316E430E326E440EA8
:1003B000336E200E346E740E356E650E366E730E0F
:1003C000376E740E386E200E396E510E3A6E3D0E39
:1003D0003B6E340E3C6E4D0E3D6E680E3E6E7A0ED8
:1003E0003F6E200E406E416A1C0E1A6E000E1B6E90
:1003F0002E0E426E2E0E436E2E0E446E2E0E456E47
:100400002E0E466E2E0E476E2E0E486E2E0E496E26
:100410002E0E4A6E2E0E4B6E2E0E4C6E2E0E4D6E06
:100420002E0E4E6E2E0E4F6E2E0E506E2E0E516EE6
:100430002E0E526E2E0E536E2E0E546E2E0E556EC6
:100440002E0E566E2E0E576E2E0E586E2E0E596EA6
:100450002E0E5A6E2E0E5B6E2E0E5C6E2E0E5D6E86
:100460005E6A420E5F6E000E606E120000010D6A41
:10047000096A086A01500010D8B4000C0150051830
:100480000A6E0ABE0D1E0B6A05AE4CEF02F0041E8A
:10049000051E042AD8B4052A01AE54EF02F0001E4E
:1004A000011E002AD8B4012A015005100A6E0ABEA6
:1004B0006CEF02F056EC04F00BB083EF02F00DAEDF
:1004C000000C001E011E002AD8B4012A081E091EB5
:1004D000082AD8B4092A000C05AE7EEF02F001BE4E
:1004E0007AEF02F00150096E0050086E016A006A4E
:1004F0005FEF02F0016A006A002A000C011E001E74
:100500000B2A5AEF02F0082AD8B4092A0450085CD2
:10051000D8A45FEF02F00550095CD8A45FEF02F0A9
:10052000096A086A002AD8B4012A01AE5FEF02F016
:100530000000FF0C12009BC0E1FF9CC0E2FF200EF8
:10054000E66E010E00019B25E16E000E9C21E26E1D
:10055000200EE66E020E9B25E16E000E9C21E26EDF
:10056000200EE66E030E9B25E16E000E9C21E26ECE
:10057000200EE66E040E9B25E16E000E9C21E26EBD
:10058000300EE66E050E9B25E16E000E9C21E26E9C
:10059000E66A040E9D6F000E006E9A51005C02E147
:1005A0009951000828E29D519B25E16E000E9C2187
:1005B000E26E0A0E046E000E056E99C000F09AC03D
:1005C00001F0F5EC04F008C000F009C001F0300EB5
:1005D000002600C0E6FF0A0E046E000E056E99C0EC
:1005E00000F09AC001F0F5EC04F000C099F001C0F1
:1005F0009AF09D07D0D712003FEC05F03FEC05F0D4
:100600003FEC05F09BC015F09CC016F099C017F0A8
:100610009AC018F099C0E9FF9AC0EAFFEF929BC018
:10062000E1FF9CC0E2FFE66A110EE124006E00C00B
:10063000E1FFE76A120E005CE16E120EE926EF9A06
:10064000EF94EF92120EE95EEF94EF9AEF92300E74
:100650000001A36F25EC04F0300E0001A36F25EC20
:1006600004F0300E0001A36F25EC04F0380E0001F9
:10067000A36F25EC04F0080E0001A36F25EC04F035
:10068000010E0001A36F25EC04F0060E0001A36F1C
:1006900025EC04F00C0E0001A36F25EC04F0010E14
:1006A000196E120000019D6B99C09EF0800E991981
:1006B000006E800E000A005C04E29D2B9951000838
:1006C0009E6F9EC09FF09AC0A0F09BC0A1F0EEEC80
:1006D00003F0040E00019C6F9C51000817E29C512E
:1006E0009A25E16E000E9B21E26E9C05006E016A68
:1006F000000E015A00509A25E96E01509B21EA6EC6
:10070000EECF00F000C0E6FF9C07E6D79AC0E1FFFD
:100710009BC0E2FF200EE66E9D5317E09C6B9C5140
:100720009A25E96E000E9B21EA6EEECF02F0025090
:10073000200A02E19C2BF3D79C079C519A25E16E7D
:10074000000E9B21E26E2D0EE66E120010D0800E80
:100750000001996F1AD0C00E996F17D0940E996F3F
:1007600014D0D40E996F11D0800E996F0ED0000165
:100770009951010AECE09951020AEDE09951030AFE
:10078000EDE09951040AEDE0EFD79A05006E99511A
:10079000002600C099F0010E196E00C0A3F025ECF0
:1007A00004F0196A00019D6B9D519B25E96E000EB6
:1007B0009C21EA6EEECF00F000520DE09D519B258A
:1007C000E96E000E9C21EA6EEECFA3F025EC04F05A
:1007D00000019D2BE9D7010E196E1200A0C0E9FFA0
:1007E000A1C0EAFF200EEE6E200EEE6E200EEE6E21
:1007F000EF6A010E0001A26F9F510908D8A0A22B39
:100800009F516308D8A0A22BED6AA25100081CE2F8
:100810000A0E046E9FC000F02DEC05F008C000F039
:1008200000C0EFFFEF509F5D006E016A000E015A9D
:100830000A0E046E000E056E36EC02F000C09FF04A
:10084000300EED26A207E1D7120015C0E9FF16C051
:10085000EAFF17C0E1FF18C0E2FFEF6A0001A353EF
:1008600000E0A3BFEF8EA3BDEF8CA3BBEF8AA3B9BB
:10087000EF88A3B7EF86A3B5EF84A3B3EF82A3B14C
:10088000EF801950010A02E1E79402D00001E784E9
:100890000001E78A6FEC05F0E79A1950010A03E1BD
:1008A0003FEC05F002D064EC05F0120000010134C9
:1008B000083609360450085E0550D8A0053C095E8C
:1008C000003601360F0E0C6E01340836093604501E
:1008D00000A072EF04F0085E0550D8A0053C095E48
:1008E00077EF04F008260550D8B0053C09260036FD
:1008F00001360C2E64EF04F000B085EF04F00450D4
:1009000008260550D8B0053C092600001200C26A2E
:10091000C00EC212C18CC18E99C000F0003600908A
:1009200000360090003600900050C212C2806AEC7F
:1009300005F0C284C2B4FED7080E026EC4CF00F028
:10094000000E016E025005E0003600900136FF0FE8
:10095000FAD7C3500012000E0112C290120099C0C3
:100960009DF09AC09EF09DC002F09EC003F0000171
:100970009D4B9E2B9BC0E9FF9CC0EAFF9B4B9C2B91
:10098000EECF00F002C0E1FF03C0E2FF00C0E6FFCF
:1009900002C0E9FF03C0EAFFEECF00F00052E3E13E
:1009A00099C000F09AC001F012001AC09FF01BC05D
:1009B000A0F013EC05F000C09AF00001996B99517A
:1009C0001A24E96E000E99BFFF0E1B20EA6EEECFCF
:1009D0009FF05CEC05F00001992B800E9919006ED8
:1009E000800E9A19005CEBE312000001086A096AA4
:1009F000100E0C6E0134083609360450085E05509E
:100A0000D8A0053C095ED8B00DEF05F004500826CB
:100A10000550D8B0053C0926D890003601360C2E7A
:100A2000FAEF04F012009FC0A1F0A0C0A2F0A1C094
:100A3000E9FFA2C0EAFF0001A14BA22BEECF00F01C
:100A40000052F5E19F51A15D006EA051A259016EC7
:100A5000010E005E000E015A12000001086B080E24
:100A60000C6E003408360450085ED8B03AEF05F03A
:100A70000826D89000360C2E31EF05F01200080E33
:100A80000B6EFF0E0A6E0B2E01D003D00A2EFED77E
:100A9000FAD71E0E0A6E0A2EFED71200816A936ADA
:100AA000010EC26E8E0EC16E110E926E826A100E13
:100AB000946EFF0E806E1200196A9FC0A3F025ECA1
:100AC00004F0010E196E1200100E0A6E0A2EFED7E7
:100AD00000001200070E0A6E0A2EFED71200000058
:100AE0001200FFFFFFFFFFFFFFFFFFFFFFFFFFFF02
:020000040030CA
:0E000000FFF9FEFEFFFFFBFFFFFFFFFFFFFF0C
:00000001FF
